:020000040800F2
:10000000709000209D010008310D00089D0A000835
:100010002D0D000895030008F511000800000000F0
:10002000000000000000000000000000910E000829
:100030004D05000800000000410D0008B501000852
:10004000B7010008B7010008B7010008B7010008B0
:10005000B7010008B7010008B7010008B7010008A0
:10006000B7010008B7010008B7010008B701000890
:10007000B7010008B7010008B7010008B701000880
:10008000B7010008B7010008B7010008B701000870
:10009000B7010008B7010008B7010008B701000860
:1000A000B7010008B7010008B7010008B701000850
:1000B000B7010008B7010008B7010008B701000840
:1000C000B7010008B7010008B7010008B701000830
:1000D000B7010008B7010008B7010008B701000820
:1000E000B7010008B7010008B7010008B701000810
:1000F000B7010008B7010008B7010008B701000800
:10010000B7010008B7010008B7010008B7010008EF
:10011000B7010008B7010008B7010008B7010008DF
:10012000B7010008B7010008B7010008B7010008CF
:10013000B7010008B7010008B7010008B7010008BF
:10014000B7010008B7010008B7010008B7010008AF
:10015000B7010008B7010008B7010008B70100089F
:10016000B7010008B7010008B7010008B70100088F
:10017000B7010008B7010008B7010008B70100087F
:10018000B7010008B7010008DFF80CD000F064F8F0
:10019000004800474D1C000870900020064880472A
:1001A00006480047FEE7FEE7FEE7FEE7FEE7FEE75C
:1001B000FEE7FEE7FEE7FEE7ED1000088901000814
:1001C000421C10F8011B0029FBD1801A704770B542
:1001D000064601F06DFC046805460A2200213046FF
:1001E00000F002F82C6070BD2DE9F04791460F46F3
:1001F00080460446002614F8015B2DB100F03EF85D
:100200000068405DC007F6D12B2D02D02D2D18D0EF
:10021000641E4A463946204600F034F827B1396852
:10022000A14201D1C7F8008071054FF002040BD53F
:100230004042002803DD01F03BFC0460A007BDE85C
:10024000F08746F48066E4E70028F8DA01F030FC35
:1002500004606FF00040F2E7064C074D06E0E068EE
:1002600040F0010394E8070098471034AC42F6D3FD
:10027000FFF78EFFEC5E00080C5F00080048704737
:100280004C5E00082DE9F05F824600780027154695
:100290008B460AF10104B946302801D09DB113E024
:1002A00014F8010B0127782803D0582801D045B154
:1002B0000AE00DB1102D07D10027102514F8010B0D
:1002C00002E0082500E00A250026B0460EE005FB06
:1002D000080005FB06F1012701EB10461FFA80F824
:1002E000B6F5803F00D3B94614F8010B294600F05B
:1002F00018F80028EBDABBF1000F05D00FB1641E2F
:1003000000E05446CBF80040B9F1000F06D001F0F0
:10031000CFFB02210160C81EBDE8F09F48EA0640FD
:10032000FAE73A2800D2303820F02002412A01D3DF
:10033000A2F13700884201D34FF0FF30704770B50B
:100340008C1810F8015B15F0070301D110F8013B80
:100350002A1106D110F8012B03E010F8016B01F807
:10036000016B5B1EF9D12B0705D40023521E0DD45F
:1003700001F8013BFAE710F8013BCB1A921C03E0AD
:1003800013F8015B01F8015B521EF9D5A142D8D3E5
:10039000002070BD00BFFEE70146302905DB39298A
:1003A00003DCA1F13000C0B27047612905DB66298A
:1003B00003DCA1F15700C0B2F6E7412905DB46296D
:1003C00003DCA1F13700C0B2EEE73720ECE7000014
:1003D00010B5394800683949884208D23648001DAE
:1003E00037490860001F00683649086001E000F0E6
:1003F000EBFD35A000F04EFD002858D035480068D0
:1004000000785B2804D133480068401C31490860FB
:10041000002404E000F0D6FA2F490855641C042C8F
:10042000F8DB2EA000F036FDA8B12A48006800785D
:100430005B2804D127480068401C26490860002436
:1004400006E000F0BFFAC1B2234808300155641C31
:10045000042CF6DB08E0FF201F490872FF211E482C
:10046000417200218172C1721FA000F013FDA8B17A
:100470001848006800785B2804D116480068401CC2
:1004800014490860002406E000F09CFAC1B212484A
:10049000001D0155641C042CF6DB0BE000200E4906
:1004A000087100210C4841718171C17102E000F0B6
:1004B0008BFD10BD00BFFCE700000E08C0D401009A
:1004C000D0000020C4000020435F49505F414444F5
:1004D00052000000EC000020E4020020435F49507D
:1004E0005F4D41534B000000435F49505F4741540B
:1004F0004500000010B500220268134B1A40CC687A
:100500000B6823434C6923438C692343CC69234301
:100510000C6A23434C6A23438C6A23434C6B23436A
:100520008C6B23431A430260426922F00702D1E92F
:100530000B3423431A4342610B6943604B68836069
:100540008B68C36010BD00003F801CF07047000046
:1005500001490860704700000C3C024070B5044639
:100560000A460026082502B909E0012A01D116022F
:1005700005E0022A01D1160201E04FF4407600F0B6
:1005800097F80546082D28D11548006820F44070DA
:100590001349086008460068304308600846006850
:1005A00020F0F80008600846006844F002010843A3
:1005B0000B4908600846006840F48030086000F08D
:1005C00077F805460648006820F0020004490860F4
:1005D0000846006820F0F8000860284670BD00005A
:1005E000103C024008201049096801F48031B1F53F
:1005F000803F01D1012015E00B49096801F010018D
:1006000009B105200EE00849096801F0EF0109B1C0
:10061000062007E00449096801F0020109B107203A
:1006200000E00820704700000C3C024003480068CE
:1006300040F000400149086070470000103C024053
:1006400030B502460C46082500F032F80546082D64
:1006500017D10D48006820F440700B490860084627
:10066000006808600846006840F0010008601470E7
:1006700000F01EF805460448006820F00100024919
:100680000860284630BD0000103C02400548006864
:1006900000F0004028B1044802490C3908600348C2
:1006A00008607047103C024023016745AB89EFCDDD
:1006B00008B508200090FFF795FF009002E0FFF7D3
:1006C00091FF00909DF800000128F8D09DF80000EF
:1006D00008BD000010B50446FFF7D8FFF320FFF770
:1006E00037FF02211820FFF739FF00201B4908605F
:1006F00025E01A480068205C7D2800D123E01748D7
:100700000068205C202800D11DE014480068205CAF
:100710000A2800D117E011480068205C0D2800D19C
:1007200011E00E4A1268A15C0C4A12680C4BD018FA
:10073000FFF786FF09480068401C08490860074821
:100740000068FF28D5D900BF04490968044A881801
:100750000021FFF775FFFFF769FF10BD9000002033
:1007600000C0000810B50446FFF790FFF320FFF724
:10077000EFFE00204549086080E045480068454993
:10078000884207D102212020FFF7E8FE082801D087
:1007900000BFFEE73E4800683F49884207D102217A
:1007A0002820FFF7DBFE082801D000BFFEE738480D
:1007B00000683A49884207D102213020FFF7CEFE77
:1007C000082801D000BFFEE731480068344988425C
:1007D00007D102213820FFF7C1FE082801D000BF51
:1007E000FEE72B4800682F49884207D102214020AC
:1007F000FFF7B4FE082801D000BFFEE724480068D8
:100800002949884207D102214820FFF7A7FE08287E
:1008100001D000BFFEE71E4800682449884207D186
:1008200002215020FFF79AFE082801D000BFFEE702
:10083000174800681749884216D3154800681C49B4
:10084000884211D21B4811490968405CFF280BD02F
:1008500018480E4A1268815C0D480068FFF7F0FEE8
:10086000082801D000BFFEE709480068401C08497D
:10087000086006480068401C044908600348006896
:10088000A042FFF47AAFFFF7D1FE10BD9000002028
:10089000E800002000000108000002080000040831
:1008A000000006080000080800000A0800000C0804
:1008B00000000E0843830020F0B50A460021002303
:1008C000002400BF3DE0012505FA01F3156805EAA3
:1008D00003049C4234D105684F000326BE40B54353
:1008E000056015794E00B5400668354305601579F9
:1008F000012D02D01579022D16D185684F000326EF
:10090000BE40B543856055794E00B5408668354395
:100910008560456801268E40B543456045689679F7
:100920008E40B6B235434560C5684F000326BE40D1
:10093000B543C560D5794E00B540C6683543C5603E
:10094000491C1029BFD3F0BDF0B5002300244D078A
:10095000ED0E02FA05F3CE1000F1200555F82650F1
:100960004E07F70E0F26BE40B543CF1000F120060C
:1009700046F82750CE1000F1200555F8265045EADC
:100980000304CE1000F1200545F82640F0BD418358
:1009900070470183704730B5024612F8010BFFF72C
:1009A000FBFC0446102C01DD002030BD1078FFF761
:1009B000F3FC0346102B01DD0020F6E703EB0410E7
:1009C000C0B2F2E710B50C48006800785D2801D18C
:1009D000002010BD08480068FFF7F9FB84B200BF93
:1009E00005480068017804480068401C024A10600D
:1009F0002C29F5D12046ECE7EC00002070B502254B
:100A00002248234908600846006800783A281BD12C
:100A100015E01F480068007853280BD11C48006877
:100A2000401C1B49086008460068FFF7D0FB0546DC
:100A3000284670BD16480068401C154908601448D7
:100A4000006800780028E4D11248114908600024A9
:100A500016E00F480068006800B90BE00C48006819
:100A600000680D49884200D90CE009480068056813
:100A70002846DEE7641C06480068001D044908603B
:100A8000082CE6D300BF2846D3E7000000C00008CA
:100A9000900000200078FF1F9999990000BFFEE7A1
:100AA00001464FF48042224B1A800A0A214B1A73E6
:100AB00000BF204A127A02F00102002AF9D01D4A32
:100AC000127B1C4B197300BF1A4A127A02F0010202
:100AD000002AF9D0174A127B0022164B1A7300BF66
:100AE000144A127A02F00102002AF9D0114A127B4C
:100AF0000122104B1A7300BF0E4A127A02F0010253
:100B0000002AF9D00B4A127B00220A4B1A7300BF4D
:100B1000084A127A02F00102002AF9D0054A107B35
:100B200000BF4FF48042024B9B1E1A8070470000AA
:100B30001A0C02400030014010B501464FF48040CD
:100B4000284B1880080A284B187300BF2648007AE3
:100B500000F001000028F9D02348007B224B1973D4
:100B600000BF2148007A00F001000028F9D01E489B
:100B7000007B00201C4B187300BF1B48007A00F05C
:100B800001000028F9D01848007B0220164B18738A
:100B900000BF1548007A00F001000028F9D0124883
:100BA000007B0020104B187300BF0F48007A00F044
:100BB00001000028F9D00C4B187B020200201873AA
:100BC00000BF0948007A00F001000028F9D0064B68
:100BD000187B02434FF48043024CA41E238010462E
:100BE00010BD00001A0C02400030014002464FF4D4
:100BF0008040214B1880100A204B187300BF1F48FB
:100C0000007A00F001000028F9D01C48007B1B4B43
:100C10001A7300BF1948007A00F001000028F9D0CB
:100C20001648007B8020154B187300BF1348007ACC
:100C300000F001000028F9D01048007B01200F4B84
:100C4000187300BF0D48007A00F001000028F9D0A9
:100C50000A48007B0948017300BF0848007A00F089
:100C600001000028F9D00548007B4FF48040024B7A
:100C70009B1E1880012070471A0C02400030014072
:100C800002464FF48040274B1880100A264B1873F9
:100C900000BF2548007A00F001000028F9D0224862
:100CA000007B214B1A7300BF1F48007A00F001003F
:100CB0000028F9D01C48007B80201B4B187300BF14
:100CC0001948007A00F001000028F9D01648007B8E
:100CD0000220154B187300BF1348007A00F0010082
:100CE0000028F9D01048007B080A0F4B187300BF8A
:100CF0000D48007A00F001000028F9D00A48007B76
:100D0000094B197300BF0848007A00F00100002861
:100D1000F9D00548007B4FF48040024B9B1E1880A1
:100D2000012070471A0C02400030014000BFFEE76E
:100D300070470000014908627047000000000E4241
:100D40007047000029B1064A12680243044B1A603A
:100D500004E0034A12688243014B1A6070470000A6
:100D60003038024029B1064A12680243044B1A6027
:100D700004E0034A12688243014B1A607047000086
:100D80004038024029B1064A12680243044B1A60F7
:100D900004E0034A12688243014B1A607047000066
:100DA0002038024029B1064A12680243044B1A60F7
:100DB00004E0034A12688243014B1A607047000046
:100DC0004438024029B1064A12680243044B1A60B3
:100DD00004E0034A12688243014B1A607047000026
:100DE0002438024021B1028842F04002028004E02F
:100DF00002884FF6BF731A400280704710B5044650
:100E00001148844208D101218014FFF7DBFF002143
:100E1000A014FFF7D7FF16E00C48844208D1012147
:100E20000014FFF7AFFF00212014FFF7ABFF0AE02B
:100E30000748844207D10121C013FFF7A3FF002117
:100E4000E013FFF79FFF10BD003001400038004065
:100E5000003C004010B50022028802F441520B8889
:100E60004C8823438C882343CC8823430C89234319
:100E70004C8923438C892343CC8923431A43028022
:100E8000838B4FF2FF74234083830B8A038210BD50
:100E90007047000002462A4800682A4B18604AE062
:100EA00028480068007800B946E0264800680078C5
:100EB000FF2800D140E02348006800787D2800D159
:100EC0003AE0204800680078222805D01D480068D4
:100ED000401C1C4B18602EE01A480068401C194B3F
:100EE0001860184600680078137898421DD10021D8
:100EF00008E0505C134B1B685B5C984200D004E038
:100F0000481CC1B2505C0028F3D100BF505C60B9EE
:100F10000C480068405C222807D10A480368C81CB6
:100F20001844084B18600120704706480068401CB0
:100F3000044B186000BFB3E700BF0020F4E70000D7
:100F4000D0000020EC00002010B503461D480360CF
:100F500033E01C480068007800B92FE019480068A9
:100F60000078FF2800D129E01648006800787D2825
:100F700000D123E01348006800780C78A04217D114
:100F800000220DE0885C0F4C24682478A04200D039
:100F900009E00C480068401C0A4C2060501CC2B29A
:100FA000885C0028EED100BF885C08B9012010BD24
:100FB00004480068401C034C2060CAE700BF0020C2
:100FC000F5E70000EC000020C0200C490870A820C4
:100FD0004870012088700220C870FF200872FF212D
:100FE0000648417200218172C172002003490871D4
:100FF0000021024841718171C1717047E4020020F3
:101000000CB50020019000903448006840F4803016
:101010003249086000BF3148006800F40030009099
:101020000198401C0190009818B90198B0F5A04FA4
:10103000F1D12A48006800F4003010B1012000907E
:1010400001E0002000900098012846D1234840305C
:10105000006840F080502149403108602048006815
:1010600040F440401E4908601C48083000681B4995
:10107000083108600846006840F4204008600846CF
:10108000006840F4A05008601648091F0860081F57
:10109000006840F08070091F086000BF0F480068BA
:1010A00000F000700028F9D040F205600E49086099
:1010B0000A480830006820F0030008490831086039
:1010C0000846006840F00200086000BF034808308E
:1010D000006800F00C000828F8D10CBD0038024070
:1010E0000070004019544007003C024010B51648FB
:1010F000006840F0010014490860002012490831DE
:10110000086011480068114908400F4908601048FC
:10111000091D0860081F006820F48020091F08606E
:10112000002009490C310860FFF76AFF4FF00060AA
:101130000849086007488030006840F4700005499D
:101140008031086010BD000000380240FFFFF6FE4D
:101150001030002408ED00E021B1028842F00102C5
:10116000028004E002884FF6FE731A400280704746
:1011700000220288184B98420ED0184B98420BD090
:10118000B0F1804F08D0164B984205D0154B9842CD
:1011900002D0154B984204D14FF68F731A404B88FA
:1011A0001A43124B984207D0114B984204D04FF685
:1011B000FF431A400B891A4302804B68C3620B88B5
:1011C0000385054B984202D0044B984201D18B7A9B
:1011D0000386012383827047000001400004014020
:1011E0000004004000080040000C004000100040D7
:1011F0000014004000BFFEE730B503461D480168FB
:101200001D4800881D4C246860830020087100BFC1
:10121000087800F001000028FAD008790B7100BFAF
:10122000087800F001000028FAD008790020087141
:1012300000BF087800F001000028FAD008790020EB
:10124000087100BF087800F001000028FAD0087982
:1012500002020020087100BF087800F00100002899
:10126000FAD008790243044C2488044D2D682C835D
:10127000104630BDB4010020B8010020B0010020AC
:1012800030B502460B461A4C2168012404EB820457
:10129000E200184C2488184D2D686C8300240C71D2
:1012A00000BF0C7804F00104002CFAD00C790B710B
:1012B00000BF0C7804F00104002CFAD00C790A71FC
:1012C00000BF0C7804F00104002CFAD00C79002443
:1012D0000C7100BF0C7804F00104002CFAD00879DE
:1012E00000BF044C2488044D2D682C8330BD0000C1
:1012F000B4010020B8010020B001002070B5024602
:101300000C461F480168012000EB8200C2001D4806
:1013100000881D4D2D6868830020087100BF087883
:1013200000F001000028FAD008790C7100BF08789D
:1013300000F001000028FAD008790A7100BF08788F
:1013400000F001000028FAD008790020087100BFE1
:10135000087800F001000028FAD008790302002084
:10136000087100BF087800F001000028FAD0087961
:101370000343044D2D88044E36683583184670BDEE
:10138000B4010020B8010020B001002030B50246B1
:101390000B461748016817480088174C246860837B
:1013A0000020087100BF087800F001000028FAD082
:1013B00008790A7100BF087800F001000028FAD00F
:1013C00008790420087100BF087800F001000028A7
:1013D000FAD008790B7100BF087800F001000028EE
:1013E000FAD00879034C2488034D2D682C8330BD36
:1013F000B4010020B8010020B001002030B5034640
:101400000A461C4801681C4800881C4C24686083FC
:101410000020087100BF087800F001000028FAD011
:1014200008790B7100BF087800F001000028FAD09D
:1014300008790420087100BF087800F00100002836
:10144000FAD00879100A087100BF087800F001008E
:101450000028FAD008790A7100BF087800F001006E
:101460000028FAD00879044C2488044D2D682C8378
:1014700030BD0000B4010020B8010020B001002000
:1014800070B503460C4619480168012000EB830043
:10149000C30017480088174D2D6868830020087125
:1014A00000BF087800F001000028FAD008790C711C
:1014B00000BF087800F001000028FAD00879181D54
:1014C000087100BF087800F001000028FAD0087900
:1014D0000A7100BF087800F001000028FAD00879EE
:1014E000034D2D88034E3668358370BDB40100204E
:1014F000B8010020B001002070B503460C461E481C
:101500000168012000EB8300C3001C4800881C4DCB
:101510002D6868830020087100BF087800F0010082
:101520000028FAD008790C7100BF087800F001009B
:101530000028FAD00879181D087100BF087800F05B
:1015400001000028FAD00879100A087100BF087855
:1015500000F001000028FAD008790A7100BF08786D
:1015600000F001000028FAD00879044D2D88044EBF
:101570003668358370BD0000B4010020B80100203A
:10158000B00100200549064A11604FF48041054A28
:1015900011600549054A116070470000000C0240C7
:1015A000B0010020B801002008300140B401002043
:1015B00010B5052203216248FFF7C6F90522042170
:1015C0005F48FFF7C1F9052211465D48FFF7BCF9F6
:1015D00002205C490871002088710220C87148719E
:1015E000082008605648FFF767F920205549086031
:1015F0005348FFF761F91020524908605048FFF73F
:101600005BF95148FFF7FAFB0020504908808880B9
:10161000C88008814FF40070488100208881C8810B
:10162000072008824FF4827048804748FFF712FC79
:1016300001214548FFF7D6FB0420424908600120FC
:10164000087100208871022048714148FFF734F981
:1016500004213F48FFF79BF94FF4404039490860A7
:101660000120087100208871022048713948FFF775
:1016700023F94FF440413748FFF78BF901203149F6
:101680000860087100208871022048713048FFF717
:1016900013F901212E48FFF77AF900202949087132
:1016A000C8714FF4006008602B48FFF705F94FF050
:1016B000C0602A49086024480C3048602848886087
:1016C0000020C86093200861002048614FF48060CA
:1016D00088610020C861086248624FF40030886267
:1016E0000020C862012008630020486388631D4809
:1016F000FEF700FF4FF0C0601849086012480C3038
:101700004860194888604020C86093200861002024
:1017100048614FF4806088610020C86108624862B7
:101720004FF4003088620020C86201200863002066
:10173000486388630B481830FEF7DCFE10BD0000DC
:1017400000040240640000200030014068020020D4
:1017500000180240000C0240001402407C020020ED
:10176000438B0020406402400001002010B5052298
:1017700003215A48FFF7E8F8052204215748FFF7EC
:10178000E3F8052211465548FFF7DEF802205449D8
:101790000871002088710220C87148710820086013
:1017A0004E48FFF789F820204D4908604B48FFF765
:1017B00083F810204A4908604848FFF77DF84948F7
:1017C000FFF71CFB0020484908808880C8800881FA
:1017D0004FF40070488100208881C881072008826A
:1017E0004FF4827048803F48FFF734FB01213D48A9
:1017F000FFF7F8FA4FF440403949086001200871BA
:1018000000208871022048713848FFF755F84FF4DE
:1018100040413648FFF7BDF80120314908600871A2
:1018200000208871022048713148FFF745F80121F6
:101830002F48FFF7ACF8002029490871C8714FF410
:10184000006008602B48FFF737F84FF0C0602A4966
:10185000086024480C304860284888600020C86030
:1018600079200861002048614FF480608861002081
:10187000C861086248624FF4003088620020C86284
:10188000012008630020486388631D48FEF732FE8C
:101890004FF0C0601849086012480C304860194881
:1018A00088604020C86079200861002048614FF4BA
:1018B000806088610020C861086248624FF400308F
:1018C00088620020C86201200863002048638863A2
:1018D0000B481830FEF70EFE10BD00000004024059
:1018E000640000200030014068020020000C02402B
:1018F00000180240001402407C020020438B0020AC
:1019000040640240BC01002000B50920FFF714F933
:1019100000BD00B50920FFF76FFC00BD10B50446FF
:101920004FF4804101EB0421491C8AB20221104688
:10193000FFF75CF900BF4FF4804202EB0422521C17
:1019400091B20846FFF7ACF80028F4D110BD10B5ED
:101950000446022201212046FFF792FD00BF01212B
:101960002046FFF78DFC0028F9D110BDF0B50446E4
:101970000F4615461E464FF4804101EB04218AB202
:1019800039461046FFF732F94FF4804101EB04214C
:10199000091D8AB229461046FFF772F94FF48041BB
:1019A00001EB042110318AB231461046FFF768F985
:1019B0004FF4804101EB0421491C8AB201211046F9
:1019C000FFF714F900BF4FF4804202EB0422521CCF
:1019D00091B20846FFF764F80028F4D1F0BDF0B5E5
:1019E00006460C4617461D46224600213046FFF7A4
:1019F00047FD3A4604213046FFF77EFD2A46102176
:101A00003046FFF779FD012211463046FFF738FDD9
:101A100000BF01213046FFF733FC0028F9D1F0BDAB
:101A200010B5044621780920FFF7E0F861780A2014
:101A3000FFF7DCF8A1780B20FFF7D8F8E1780C204D
:101A4000FFF7D4F821790D20FFF7D0F861790E2047
:101A5000FFF7CCF810BD10B5044621780920FFF738
:101A600095FC61780A20FFF791FCA1780B20FFF725
:101A70008DFCE1780C20FFF789FC21790D20FFF720
:101A800085FC61790E20FFF781FC10BD0FB408467C
:101A900010B5064A02A900F01EF8044602A900206B
:101AA00000F02AF8204610BC5DF814FBF91A000873
:101AB000004870473C02002002E008C8121F08C11D
:101AC000002AFAD170477047002001E001C1121FBF
:101AD000002AFBD170472DE9F04116460F46044617
:101AE000002503E03946B047641C6D1C20780028AF
:101AF000F8D12846BDE8F0810A68531C0B601070CD
:101B0000704710B504464FF4804101EB0421491C95
:101B10008AB210211046FFF769F800BF4FF48042E7
:101B200002EB0422521C91B20846FEF7B9FF0028CE
:101B3000F4D14FF4804101EB0421891C8AB2FF21CA
:101B40001046FFF753F810BD10B5044610220121CE
:101B50002046FFF795FC00BF01212046FFF790FBD0
:101B60000028F9D1FF2202212046FFF789FC10BD91
:101B700010B504464FF4804101EB0421491C8AB2A0
:101B800008211046FFF732F800BF4FF4804202EB05
:101B90000422521C91B20846FEF782FF0028F4D1BD
:101BA00010BD10B50446082201212046FFF768FC4D
:101BB00000BF01212046FFF763FB0028F9D110BDCB
:101BC0000146CA0202F5404290B270470146CA027D
:101BD00002F5004290B2704710B504464FF48042BF
:101BE00002EB0422263291B20846FEF7A5FF10BD93
:101BF00010B5044626212046FFF780FB10BD10B526
:101C000004464FF4804202EB0422D21C91B20846F3
:101C1000FEF746FF10BD10B5044603212046FFF72E
:101C20002FFB10BD10B504464FF4804202EB042296
:101C3000203291B20846FEF77FFF10BD10B5044672
:101C400020212046FFF75AFB10BD0000FE488068A7
:101C500040F48050FC4988600121FC48FFF772F88D
:101C6000012141F21000FFF79DF80121F848FFF72C
:101C700079F80120FFF75EF8F648006840F48070BC
:101C8000F44908600020F44908710120C8717F20E0
:101C90000860F248FEF710FEF14C282503E0641EB0
:101CA0000CB96D1EEE4CED48006900F0100008B94B
:101CB000002DF4DC35B90020EA4988600120EA49AA
:101CC000088067E00020E8490880E6488068E74926
:101CD000884212D10020E34988604CF6CC40E449A8
:101CE000086045F255500860012048601020886067
:101CF0004AF6AA20086000BFFEE7DA488068DD499E
:101D0000884246D0DC480068DC490840B0F1005FFA
:101D10003FD1D948006ADA490860D748406AD949B2
:101D20000860D5483030D8490860D5480068B0F51B
:101D3000503F00D92EE0D3480068D0B10120D349EC
:101D4000886000240AE0D04800680068CF49086035
:101D5000CD480068001DCC490860641CC848006874
:101D60008442F0D3C9480068C6490968884200D057
:101D700010E0C1484068C649086008460068C54987
:101D80000860BD49086880F3088800BFC148006842
:101D9000804700BF0220B0490871002088710220EE
:101DA000C87148714FF4E0500860BB48FEF784FDED
:101DB00006220A21B848FEF7C7FD06220B21B648C5
:101DC000FEF7C2FD06220C21B348FEF7BDFD4FF41D
:101DD0004050A1490860012008710020887102204C
:101DE0004871AE48FEF768FDAD48FFF707F80020E0
:101DF000AC4908808880C88008814FF40070488111
:101E0000282088810020C881072008824FF4827032
:101E10004880A348FFF71EF80121A148FEF7E2FF22
:101E20001420A14908702820487050208870A120F3
:101E3000C87042200871852048710A2088711420DA
:101E4000C8712820087250204872A1208872422050
:101E5000C872852008730A2048734FF480518F4858
:101E6000FEF795FD4FF400518C48FEF790FD8C482D
:101E70000C3000888D490860002089490C310880A9
:101E800000BF87480830008800F001000028F8D023
:101E900083480C300088854908604FF400517F4822
:101EA000FEF777FD002405E07D48083000887F4973
:101EB0000860641CB4F5FA7FF6DB4FF400517748F4
:101EC000FEF765FD4FF480517448FEF762FD002572
:101ED0002CE073480C300088744908607248405DFB
:101EE0006F490C31088000BF6D480830008800F051
:101EF00001000028F8D06A480C3000886B4908605F
:101F00004FF400516548FEF744FD002405E06448A5
:101F10000830008865490860641CB4F5FA7FF6DB78
:101F20004FF400515D48FEF732FD6D1C0E2DD0DBE5
:101F30004FF480515948FEF72AFD00215848FEF71A
:101F400051FF5748FEF75AFF0020564908804FF4CA
:101F5000006088800020C88008814FF400704881AC
:101F6000282088810020C881072008824FF48270D1
:101F700048804B48FEF76EFF01214948FEF732FFCB
:101F80000020354908710120C8717F20086033485E
:101F9000FEF792FC314801697F20884320F0100051
:101FA000434908600020434908604148007800F038
:101FB0000100002846D04048404908604048414957
:101FC0000860414841490860414842490860424828
:101FD0004249086042484349086043484349086011
:101FE00043484449086044484449086044484549D6
:101FF00008604548454908604548464908604648E4
:1020000046490860464847490860474847490860CC
:10201000474848490860484848490860484849498D
:1020200008604948494908602248006840F48040F7
:1020300020490860FFF7A6FA1E48006840F4805067
:102040001C4985E086E00000002004E07F10640069
:102050000180001000700040640000200010024069
:1020600040420F00004002408E000020009125FCFD
:102070000030004071554812000001080000FE2F9A
:1020800080000020840000208800002000300240F2
:10209000F4000020F000002000080240000C024084
:1020A000003C004068020020438300209000002094
:1020B000F8000020FC000020A31B000818000020EE
:1020C0005D2D00081C0000203D320008200000208B
:1020D000C92F000824000020491B00082800002008
:1020E000DF1900082C0000204F19000830000020E4
:1020F000F11B0008340000206B3400083800002079
:10210000571A00083C00002023330008400000203C
:102110000F34000844000020573300084800002016
:102120008F3300084C00002073330008500000205B
:102130001319000854000020C33300085800002081
:102140003D1C00085C000020171C000860000020F7
:10215000086040E0F348F4490860F448F449086036
:10216000F448F5490860F548F5490860F548F6492E
:102170000860F648F6490860F648F7490860F748ED
:10218000F7490860F748F8490860F848F8490860D6
:10219000F848F9490860F948F9490860F948FA49E6
:1021A0000860FA48FA490860FA48FB490860FB48A9
:1021B000FB490860FB48FC490860FC48FC49086092
:1021C000FC48FD490860FD48006840F48050FB4928
:1021D0000860FFF7D7F9FA48008810B1FEF7F4FE5F
:1021E00001E0FEF7F5F8F7488068F74988420CD11E
:1021F000F448C06848B1F348C068F4490860F14841
:1022000040698860EF48006948600020ED498860B7
:10221000FEF7F4FBEE490860EE4800684008EE491E
:10222000B0FBF1F0401EED49088000204880401EC0
:1022300048600020088188724FF08040FEF798FFC8
:1022400001218807FEF788FFDC48008800F4804001
:1022500010B1FFF78BFA01E0FFF7AAF90121E0487E
:10226000FEF795FB00204FF0804148620846406A27
:10227000DC490844DC49086000BF4FF08040406AF8
:10228000D94909688842F8D30121D548FEF781FB76
:1022900000204FF0804148620846406AD349084414
:1022A000D149086000BF4FF08040406ACE490968BC
:1022B0008842F8D30020CE490860C5480068CA4962
:1022C00008600846006842F21071B0FBF1F00404A7
:1022D000C5480068B0FBF1F201FB1200C24908607A
:1022E000084600684FF47A71B0FBF1F004EB00345B
:1022F000BD480068B0FBF1F201FB1200BA4908606A
:10230000084600686421B0FBF1F004EB0024B648F5
:102310000068B0FBF1F201FB1200B3490860084607
:1023200000680A21B0FBF1F004EB0014AE4800682D
:10233000B0FBF1F201FB1200AB49086008460068EF
:1023400020440860FA20AB490870CE204870102065
:102350008870A5480068000CC870A3480088000A6F
:102360000871A14800784871084681490968884782
:1023700096488D490968884794480830804909681B
:1023800088479248001D7C490968884741F2883097
:102390007F490968884707207F490968884772484C
:1023A000006880474CF6CC409349086045F2555090
:1023B0000860042048604FF47A7088604AF6AA20CA
:1023C000086000204FF0804148620846406A854915
:1023D00008448A490860002089490860ECE34AF60D
:1023E000AA20854908604007406A844909688842F4
:1023F0007ED900204FF0804148620846406A794902
:1024000008447E4908607E480068401C7C4908609A
:102410000846006840F6B83188420FD94CF6CC40E7
:102420007549086045F25550086001204860102049
:1024300088604AF6AA20086000BFFEE7714800687D
:10244000401C704908600846007800F0040008B39A
:102450004FF400516C48FEF79AFA6C4800886249C4
:10246000086045F255506949088000BF6748001F61
:10247000008800F001000028F8D0644800885A491C
:1024800008604FF400516048FEF783FA00205D4970
:10249000086024E04FF400515B48FEF778FA5B488F
:1024A0000088514908605A48008820B14AF6AA209D
:1024B0005649088002E000205449088000BF534874
:1024C000001F008800F001000028F8D04F48008865
:1024D000454908604FF400514B48FEF75AFA4C4802
:1024E0000088B0F57A7F03DD49480088401E00E08F
:1024F00016E04749088008460088B0F57A7F0FDC6F
:102500004CF6CC403C49086045F25550086001202B
:102510004860102088604AF6AA20086000BFFEE7E5
:1025200078E00000711B000818000020132D00083F
:102530001C000020FB310008200000206D2E000848
:1025400024000020031B0008280000206D1900084B
:102550002C0000201D19000830000020D91B0008A5
:10256000340000203534000838000020211A00080B
:102570003C000020FD32000840000020E933000844
:10258000440000204933000848000020813300083F
:102590004C00002065330008500000200919000895
:1025A000540000209D33000858000020251C00081E
:1025B0005C000020FF1B000860000020FC000020E1
:1025C0008E0000200040024071554812E4020020B5
:1025D000780000200000002040420F004002002050
:1025E00000180240A08601009000002020A10700F2
:1025F000D8000020DC0000200030004094000020C3
:10260000980000209C000020000C02400C3C004080
:102610008C000020F848006800287DD0F64800684B
:10262000C01E062877D2DFE800F0EAE976A5E803C5
:10263000F2A1F548FEF788FCF0B3FEF727F8F32087
:10264000FDF786FF02215820FDF788FFFDF7EEFF1A
:10265000EE49EF48FFF71AFAED48FDF7B1FDED49F5
:1026600008600846008882B2E9490720EA4B1B68E7
:10267000984700204FF08041486200BF4FF08040F3
:10268000406A4CF250318842F8D30720E349096888
:10269000884700204FF08041486200BF4FF08040E3
:1026A000406A4CF250318842F8D30020DC498860FF
:1026B0004CF6CC40DB4900E00CE0086045F2555098
:1026C000086001204860102088604AF6AA2008604F
:1026D00000BFFEE7D4A1CC48FEF736FCE8B1FDF719
:1026E000D5FFF320FDF734FF02214820FDF736FF28
:1026F000FDF79CFFC549C648FFF7C8F9C448FDF778
:102700005FFDC44908600320BB4908600020C94937
:102710000860C9490860C5E1C5E1C8A1BA48FEF72B
:1027200013FCA8B1C8480068FDF7D4FFB749B84802
:10273000FFF7ACF9B648FDF743FDB6490860032042
:10274000AD4908600020BB490860BB490860A9E1A9
:10275000BE484068BE4908600020B6490860BB48D2
:10276000C068BA494968401AAA4908600320A249CA
:10277000086097E1B7480088F0BBB7A1A248FEF710
:10278000E3FB002871D0A149A148FFF77FF9A048D9
:10279000FDF716FDA84908600846008882B29C49EA
:1027A00007209D4B1B68984700204FF080414862EE
:1027B00000BF4FF08040406A4CF250318842F8D35D
:1027C000072096490968884700204FF080414862F9
:1027D00000BF4FF08040406A4CF250318842F8D33D
:1027E00000208F4988604CF6CC408E49086045F245
:1027F00055500860012003E00AE043E046E1D1E0E3
:102800004860102088604AF6AA20086000BFFEE7F2
:102810007D488D49086000241BE08B4800680078E3
:10282000212804D188480068401C874908608648F0
:10283000006800787D2800D10EE083480068FEF72C
:10284000AAF87349085580480068801C7E490860D2
:10285000641CB4F5806FE0DB00BF14B12046FDF7C7
:1028600081FF4FF47F707B4908807E496848FFF7FD
:102870000DF96748FDF7A4FC6F49086004205E4924
:1028800008600FE173480088B8BB77A15E48FEF787
:102890005BFB98B36C48006800783A2803D00520A9
:1028A00055490860FEE068480068401C66490860B9
:1028B00068480088401C6749088063480068FEF744
:1028C0006AF800066B4908605F480068801C5E4932
:1028D000086008460068FEF75EF86649096841EA44
:1028E00000406449086058480068801C56490860E8
:1028F00060480068604908600CE007E0FFE70020DE
:102900004D49086005203C4908604AE03E484E4970
:10291000086000BF002416E04B48006800787D285E
:1029200004D0494800680078212800D10EE04648CC
:102930000068FEF730F83649085543480068801CA7
:1029400041490860641CB4F5806FE5DB00BF14B139
:102950002046FDF707FF3C480068401C3A490860E4
:10296000002046490860012023490860002415E042
:1029700035480068007828B133480068007822495B
:10298000085500E00CE030480068401C2E49086003
:102990003A480068401C39490860641CFA2CE7DB9F
:1029A00000BF7FE036480068B0F5FA7F6DD9224855
:1029B0000068F0B9002414E01E4800681549096851
:1029C00088420CD2224800681A490968405C1049C4
:1029D000085518480068401C1649086000E003E0EC
:1029E000641CB4F5967FE7DB00BF1CB1124804609D
:1029F0004BE04AE046E00000A8000020436C65611F
:102A000072436F6E6600000044030020505E0008B1
:102A100043830020B8000020200000201800002080
:102A20000040024000300040436C65617243616CBD
:102A300063000000B4000020AC0000205365745017
:102A40003D7B313739360000EC000020B85D0008CE
:102A5000CC0000208C00002072756E6D61696E3DA7
:102A60007B000000A45E00084669726D4845583D31
:102A70007B000000E4000020E8000020A40000200B
:102A8000C800002004207A4908600BE079480068FB
:102A9000B0F5006F05D17848006810B90520744979
:102AA000086000BF00BF072074490968884790B1DB
:102AB000132804D0172829D01C280BD11AE007208E
:102AC0006F490968884700206E4908606E490860B0
:102AD00067490860C9E000235022012107206B4E9E
:102AE0003668B04700206749086067490860604958
:102AF0000860BAE0072066490968884700206149F4
:102B00000860614908605A490860AEE007206149E1
:102B100009688847574908605548006806287CD2EC
:102B2000DFE800F00304A284859600BF07205A491D
:102B3000096888475949086008460068D8B30846BC
:102B40000068642801D9642008605448008882B273
:102B500053484C4B1B68C1180720524B1B689847C1
:102B60004348006830BB4E48007847280FD14C4896
:102B7000407845280BD14A488078542807D14848E6
:102B8000C078202803D108203949086018E044485B
:102B90000078502811D1424840784F280DD1404844
:102BA0008078532809D13E48C078542805D10120A7
:102BB0002F49086004E038E058E005202C490860FF
:102BC0002B480068012819D1002413E02D48006823
:102BD00020443349085C212802D07D2808D103E035
:102BE00007202349086003E006202149086000BF50
:102BF00000BF641C294800688442E7D3214800686C
:102C00002649096808441F490860002024491D4AD4
:102C1000126888541B48006800E025E047F2FD7107
:102C2000884202D90520124908601DE000BF124801
:102C3000006860B11048008882B21B4907201B4B16
:102C40001B68984700200B4908600B4908600BE09F
:102C500007200F490968884700200A4908600A4987
:102C600008600349086000BF00BF00BFFFF7B7BBA3
:102C7000A8000020C8000020AC0000206000002058
:102C800030000020A4000020B00000202C00002014
:102C9000180000205C00002034000020800000208C
:102CA000440300201C00002043830020200000205B
:102CB0002DE9F0478246894616461C46C9F30A08A4
:102CC0005046FEF77DFF00EB080508EB0400B0F569
:102CD000006F16DDC8F500618FB2ABB23A463146DF
:102CE000184600F0C3FB3E44E11B8FB25046FEF78E
:102CF00067FF05462B463A463146184600F0B6FBBC
:102D000005E0ABB222463146184600F0AFFBBDE805
:102D1000F087F0B504460E4615460027002D1BDD52
:102D20002A463146204600F07FF84FF4804101EBFF
:102D30000421491C8AB240211046FDF757FF00BF0D
:102D40004FF4804202EB0422521C91B20846FDF778
:102D5000A7FE0028F4D12F463846F0BD2DE9F043F8
:102D600081460F4615462D490C6828214846FEF736
:102D7000C5FA06462A4800882A490968488330125D
:102D8000207100BF207800F001000028FAD02079DF
:102D9000267100BF207800F001000028FAD02079C9
:102DA0004FEA8900C01C002101EBC000207100BF68
:102DB000207800F001000028FAD020794FF00008B8
:102DC0000EE00020207100BF207800F001000028F4
:102DD000FAD0207938707F1C08F101001FFA80F8C2
:102DE000A845EEDB0E4909880E4A12681183711955
:102DF0008EB2324628214846FEF77EFB4022012152
:102E00004846FEF73DFB00BF01214846FEF738FA71
:102E10000028F9D12846BDE8F0830000B401002065
:102E2000B8010020B0010020F0B504460E4615465A
:102E30004FF4804202EB0422283291B20846FDF79B
:102E40007BFE07462B46324639462046FFF730FFC9
:102E500079198FB24FF4804101EB042128318AB2F5
:102E600039461046FDF70CFFF0BD00002DE9FC438C
:102E700004468946154698464FF4804202EB0422E8
:102E8000283291B20846FDF757FE07464FF48042BC
:102E900002EB042291B20846FDF702FE00F00700A3
:102EA000022804D003282BD0042856D144E008235C
:102EB0006A4639462046FFF7FBFE07F1080087B255
:102EC0009DF8000028709DF8010068709DF80200D0
:102ED000A8709DF80300E8709DF80400A8F80000B1
:102EE0009DF8050098F8001000EB0120A8F80000FC
:102EF0009DF806609DF8070000EB062086B22DE0E5
:102F000006236A4639462046FFF7D2FEB81D87B22F
:102F10009DF8000028709DF8010068709DF802007F
:102F2000A8709DF80300E8709DF804609DF8050006
:102F300000EB062086B211E002236A46394620469D
:102F4000FFF7B6FEB81C87B29DF800609DF801003F
:102F500000EB0620801E86B200E000BF00BFB6F581
:102F6000007F06DA33464A4639462046FFF7A0FE80
:102F700000E00026B9198FB212490F804FF480414A
:102F800001EB042128318AB239461046FDF778FE5C
:102F90004FF4804101EB0421491C8AB240211046C4
:102FA000FDF724FE00BF4FF4804202EB0422521CC6
:102FB00091B20846FDF774FD0028F4D13046BDE813
:102FC000FC830000AC0100202DE9FF4B8146154633
:102FD000984676490C6828214846FEF78FF907463F
:102FE000734800887349096848833812207100BF0C
:102FF000207800F001000028FAD02079277100BF66
:10300000207800F001000028FAD020794FEA8900EA
:10301000C01C002101EBC000207100BF207800F02F
:1030200001000028FAD020790020207100BF20780C
:1030300000F001000028FAD02079287000202071CB
:1030400000BF207800F001000028FAD020796D1C24
:1030500028700020207100BF207800F001000028B7
:10306000FAD020796D1C28700020207100BF2078D4
:1030700000F001000028FAD020796D1C2870002093
:10308000207100BF207800F001000028FAD02079DC
:10309000A8F800000020207100BF207800F0010097
:1030A0000028FAD0207998F8001000EB0120A8F849
:1030B00000000020207100BF207800F001000028EF
:1030C000FAD0207906460020207100BF207800F059
:1030D00001000028FAD0207900EB062086B234489F
:1030E000008834490968088307F1080087B2B6F5FB
:1030F000007F40DC2E4800882E490968488338123A
:10310000207100BF207800F001000028FAD020795B
:10311000277100BF207800F001000028FAD0207944
:103120004FEA8900C01C002101EBC000207100BFE4
:10313000207800F001000028FAD020794FF0000B31
:1031400012E00020207100BF207800F0010000286C
:10315000FAD020792179019801700198401C0190E2
:103160000BF101001FFA80FBB345EADB1048008831
:10317000104909680883B9198FB23A462821484690
:10318000FEF7BAF9402201214846FEF779F900BF5F
:1031900001214846FEF774F80028F9D1B6F5007F02
:1031A00002DD04B0BDE8F08B3046FAE7B401002040
:1031B000B8010020B0010020F0B504460F461546C6
:1031C0004FF4804202EB0422243291B20846FDF70C
:1031D000B3FC06462B4632463946204600F0FAF943
:1031E00071198EB24FF4804101EB042124318AB26F
:1031F00031461046FDF744FDF0BD70B504460D465E
:103200001646324629462046FFF7D6FF4FF4804146
:1032100001EB0421491C8AB220211046FDF7E6FC8F
:1032200000BF4FF4804202EB0422521C91B20846C8
:10323000FDF736FC0028F4D170BD00002DE9F04305
:103240008046894617462A490C6824214046FEF7E5
:1032500055F80546274800882749096848832812F9
:10326000207100BF207800F001000028FAD02079FA
:10327000257100BF207800F001000028FAD02079E5
:103280004FEA8800801C042101EBC000207100BFC0
:10329000207800F001000028FAD0207900260AE00A
:1032A00019F80600207100BF207800F00100002806
:1032B000FAD02079761CBE42F2DB0E4909880E4A0C
:1032C00012681183E9198DB22A4624214046FEF77F
:1032D00013F9202201214046FEF7D2F800BF012158
:1032E0004046FDF7CDFF0028F9D1BDE8F08300008E
:1032F000B4010020B8010020B001002010B5044640
:1033000021780120FDF772FC61780220FDF76EFC48
:10331000A1780320FDF76AFCE1780420FDF766FC44
:1033200010BD10B5044621780120FEF72FF8617812
:103330000220FEF72BF8A1780320FEF727F8E178AA
:103340000420FEF723F810BD10B5044621460020E6
:10335000FDF74CFC10BD10B5044621460020FEF7D9
:1033600015F810BD10B5044621461920FDF73EFCA6
:1033700010BD10B5044621461B20FEF707F810BD0E
:1033800010B5044621461720FDF77AFC10BD10B594
:10339000044621461920FEF731F810BD10B5044649
:1033A00021780F20FDF722FC61781020FDF71EFC2C
:1033B000A1781120FDF71AFCE1781220FDF716FC28
:1033C00010BD10B5044621780F20FDF7DFFF6178AE
:1033D0001020FDF7DBFFA1781120FDF7D7FFE17882
:1033E0001220FDF7D3FF10BD10B50446217805204B
:1033F000FDF7FCFB61780620FDF7F8FBA1780720BC
:10340000FDF7F4FBE1780820FDF7F0FB10BD10B5E7
:10341000044621780520FDF7B9FF61780620FDF705
:10342000B5FFA1780720FDF7B1FFE1780820FDF78F
:10343000ADFF10BD10B5002414E04FF4804101EB46
:1034400004211F318AB202211046FDF7CFFB4FF451
:10345000804101EB04211E318AB202211046FDF7A2
:10346000C5FB641C082CE8DB10BD704770B5034633
:103470000C4600214FF48040264D28805818000A41
:10348000254D287300BF2448007A00F00100002871
:10349000F9D02148007B58181F4D287300BF1E48E3
:1034A000007A00F001000028F9D01B48007BC2F32D
:1034B0000620194D287300BF1748007A00F001005C
:1034C0000028F9D01448007B134D2A7300BF12481E
:1034D000007A00F001000028F9D00F48007B00219D
:1034E0000EE000200C4D287300BF0B48007A00F05E
:1034F00001000028F9D0084D287B6054481C81B297
:103500009142EEDB4FF48045024EB61E35801046E8
:1035100070BD00001A0C02400030014070B5034637
:103520000C4600210AB9002070BD4FF48040274DA1
:1035300028805818000A264D287300BF2448007AB6
:1035400000F001000028F9D02148007B5818204DD8
:10355000287300BF1E48007A00F001000028F9D04F
:103560001B48007BC2F3062040F08000184D2873F2
:1035700000BF1748007A00F001000028F9D0144875
:10358000007B134D2A7300BF1148007A00F0010040
:103590000028F9D00E48007B00210DE0605C0C4D46
:1035A000287300BF0A48007A00F001000028F9D013
:1035B0000748007B481C81B29142EFDB4FF4804505
:1035C000024EB61E35801046AEE700001A0C0240CF
:1035D000003001402DE9F0478246884691461C465E
:1035E000C9F30A075046FEF7F1FAC5193819B0F5C4
:1035F000006F16DDC7F500618EB2ABB232464146B0
:103600001846FFF78BFFB044A11B8EB25046FEF761
:10361000DDFA05462B46324641461846FFF77EFF47
:1036200005E0ABB2224641461846FFF777FFBDE8FA
:10363000F087000053494E44303A32352E31312E56
:10364000323031372032303A3031003C21444F4360
:10365000545950452068746D6C3E3C68746D6C3EE6
:103660003C686561643E3C6D6574612063686172AD
:103670007365743D5554462D383E3C7469746C65D1
:103680003ED09ED0B1D0BDD0BED0B2D0BBD0B5D090
:10369000BDD0B8D0B520D0BFD180D0BED0B3D180FE
:1036A000D0B0D0BCD0BCD18B20D0BAD0BED0BDD190
:1036B00082D180D0BED0BBD0BBD0B5D180D0B03C01
:1036C0002F7469746C653E3C7374796C65207479F1
:1036D00070653D746578742F6373733E2A7B6D61EA
:1036E0007267696E3A303B70616464696E673A3044
:1036F0003B626F782D73697A696E673A626F7264A4
:1037000065722D626F787D626F64797B666F6E740F
:103710002D73697A653A2E3735656D3B666F6E7429
:103720002D66616D696C793A417269616C2C4865EE
:103730006C7665746963612C73616E732D73657249
:1037400069663B636F6C6F723A233333333B6D6151
:103750007267696E3A31656D7D6469767B6D617201
:1037600067696E3A31656D20303B6C696E652D6816
:1037700065696768743A313530257D68317B6D61E4
:103780007267696E3A3020302031656D3B666F6E2E
:10379000742D73697A653A323030257D68312C6832
:1037A000327B666F6E742D7765696768743A343062
:1037B000307D68327B6D617267696E3A32656D206B
:1037C000302031656D3B666F6E742D73697A653A92
:1037D000313530257D696E7075747B6D61726769F6
:1037E0006E3A302032656D3B70616464696E673A91
:1037F00035707820313270783B626F726465723A4E
:1038000031707820736F6C696420236262623B665A
:103810006F6E743A696E68657269743B6C696E6547
:103820002D6865696768743A6E6F726D616C3B6391
:103830006F6C6F723A233434347D696E7075743AEC
:10384000666F6375737B626F726465722D636F6CF4
:103850006F723A233032383864317D627574746F18
:103860006E7B70616464696E673A367078203132BD
:1038700070783B6261636B67726F756E643A233078
:1038800032383864313B636F6C6F723A2366666618
:103890003B626F726465723A6E6F6E653B666F6E07
:1038A000743A696E68657269743B6C696E652D68FF
:1038B00065696768743A6E6F726D616C3B6F7574A1
:1038C0006C696E653A6E6F6E657D627574746F6E4D
:1038D0003A686F7665727B6261636B67726F756E53
:1038E000642D636F6C6F723A233032393865613BF7
:1038F000626F782D736861646F773A302031707829
:1039000020337078207267626128302C302C302C84
:103910002E3132292C30203170782032707820728C
:1039200067626128302C302C302C2E3234293B63D6
:103930007572736F723A706F696E7465727D6275BD
:1039400074746F6E3A6163746976657B6261636BF0
:1039500067726F756E642D636F6C6F723A233032CD
:10396000373862383B626F782D736861646F773ADD
:1039700030202D3170782033707820726762612892
:10398000302C302C302C2E3132292C30202D31701F
:103990007820327078207267626128302C302C30A9
:1039A0002C2E3234297D627574746F6E3A3A2D6D07
:1039B0006F7A2D666F6375732D696E6E65727B62AB
:1039C0006F726465723A307D617B636F6C6F723ABF
:1039D000233232323B746578742D6465636F726193
:1039E00074696F6E3A6E6F6E657D23666163746F86
:1039F00072792D646174617B646973706C61793A6A
:103A00006E6F6E657D23666163746F72792D64617C
:103A10007461206C6162656C7B646973706C617940
:103A20003A696E6C696E652D626C6F636B3B77698A
:103A30006474683A383070787D23666163746F729D
:103A4000792D6461746120696E7075747B77696427
:103A500074683A33303070783B6D617267696E3AE2
:103A6000302031656D203020307D23666163746FB6
:103A700072792D737472696E67732D6C6973747BC0
:103A8000706F736974696F6E3A6162736F6C75748D
:103A9000653B6C6566743A34363570783B746F708C
:103AA0003A32343070783B70616464696E673A31E1
:103AB0003070783B6261636B67726F756E642D6303
:103AC0006F6C6F723A236565657D23666163746F01
:103AD00072792D737472696E67732D6C69737420BB
:103AE0006C697B6C6973742D7374796C652D747952
:103AF00070653A6E6F6E653B70616464696E673ABB
:103B000035707820303B626F726465722D626F741D
:103B1000746F6D3A31707820736F6C696420236222
:103B200062623B637572736F723A706F696E74652F
:103B3000727D237374617475737B636F6C6F723AFB
:103B40007265643B666F6E742D73697A653A3135C0
:103B500030253B746578742D616C69676E3A6365D6
:103B60006E7465727D23696E7374616C6C7B7669AB
:103B7000736962696C6974793A68696464656E7DB9
:103B80003C2F7374796C653E3C2F686561643E3CE4
:103B9000626F64793E3C68313ED0A0D0B5D0B6D0DB
:103BA000B8D0BC20D0BED0B1D0BDD0BED0B2D0BB7A
:103BB000D0B5D0BDD0B8D18F20D0BFD180D0BED0AD
:103BC000B3D180D0B0D0BCD0BCD18B20D0BAD0BEC5
:103BD000D0BDD182D180D0BED0BBD0BBD0B5D1803A
:103BE0003C6120687265663D6A61766173637269E3
:103BF00070743A766F69642830293B2069643D66A9
:103C00006163746F72792D646174612D73686F776D
:103C10003ED0B03C2F613E3C2F68313E3C6469761B
:103C20003E3C627574746F6E20747970653D627588
:103C300074746F6E2069643D65786974207469746A
:103C40006C653D22D092D18BD0B9D182D0B820D032
:103C5000B8D0B720D180D0B5D0B6D0B8D0BCD0B015
:103C600020D0BFD180D0BED0B3D180D0B0D0BCD016
:103C7000BCD0B8D180D0BED0B2D0B0D0BDD0B8D139
:103C80008F223ED092D18BD0B9D182D0B820D0B87B
:103C9000D0B720D180D0B5D0B6D0B8D0BCD0B0206D
:103CA000D0BED0B1D0BDD0BED0B2D0BBD0B5D0BDCB
:103CB000D0B8D18F20D0BFD180D0BED0B3D180D0EA
:103CC000B0D0BCD0BCD18B3C2F627574746F6E3E8B
:103CD0003C2F6469763E3C6469762069643D666188
:103CE00063746F72792D646174613E3C68323ED0BA
:103CF000A3D181D182D0B0D0BDD0BED0B2D0BAD005
:103D0000B020D0B7D0B0D0B2D0BED0B4D181D0BA6C
:103D1000D0B8D18520D0B4D0B0D0BDD0BDD18BD15A
:103D2000853C2F68323E3C6469763E3C6C6162653E
:103D30006C20666F723D666163746F72792D646189
:103D400074612D70773ED09FD0B0D180D0BED0BBF3
:103D5000D18C3A3C2F6C6162656C3E3C696E70752B
:103D60007420747970653D746578742069643D666B
:103D70006163746F72792D646174612D70773E3C5C
:103D80002F6469763E3C6469763E3C6C6162656C8A
:103D900020666F723D666163746F72792D64617421
:103DA000612D7365723ED0A1D0B5D1802FD0BD3AC0
:103DB0003C2F6C6162656C3E3C696E70757420745A
:103DC0007970653D746578742069643D66616374DB
:103DD0006F72792D646174612D7365723E3C6275FA
:103DE00074746F6E20747970653D627574746F6E53
:103DF0002069643D666163746F72792D64617461DA
:103E00002D7365722D696E633E2B3C2F6275747441
:103E10006F6E3E3C2F6469763E3C6469763E3C6C36
:103E20006162656C20666F723D666163746F727962
:103E30002D646174612D7374723ED0A1D182D180E2
:103E4000D0BED0BAD0B03A3C2F6C6162656C3E3CBB
:103E5000696E70757420747970653D74657874202E
:103E600069643D666163746F72792D646174612D5C
:103E70007374723E3C627574746F6E2074797065F1
:103E80003D627574746F6E2069643D666163746F22
:103E900072792D646174612D7374722D6C69737401
:103EA0003E266C743B2D2D2D3C2F627574746F6E05
:103EB0003E3C2F6469763E3C6469763E3C6C6162B0
:103EC000656C20666F723D666163746F72792D64F4
:103ED0006174612D73656E643E3C2F6C6162656C2C
:103EE0003E3C627574746F6E20747970653D6275C6
:103EF00074746F6E2069643D666163746F72792DAE
:103F0000646174612D73656E643ED0A3D181D182EA
:103F1000D0B0D0BDD0BED0B2D0B8D182D18C3C2FE1
:103F2000627574746F6E3E3C2F6469763E3C2F64FC
:103F300069763E3C68323ED092D0BED181D181D1EB
:103F400082D0B0D0BDD0BED0B2D0BBD0B5D0BDD065
:103F5000B8D0B520D0BAD0BED0BDD182D180D0BE2D
:103F6000D0BBD0BBD0B5D180D0B03C2F68323E3C66
:103F70006469763E3C627574746F6E207479706506
:103F80003D627574746F6E2069643D636C65617227
:103F90002D63616C63207469746C653D22D0A3D07D
:103FA000B4D0B0D0BBD0B8D182D18C20D0BFD1801A
:103FB000D0BED0B3D180D0B0D0BCD0BCD18320D0C3
:103FC000B4D0BED180D0B0D181D187D0B5D182D08C
:103FD000B0223ED0A3D0B4D0B0D0BBD0B8D182D123
:103FE0008C20D0BFD180D0BED0B3D180D0B0D0BCD7
:103FF000D0BCD18320D0B4D0BED180D0B0D181D1BB
:1040000087D0B5D182D0B03C2F627574746F6E3E8C
:10401000203C627574746F6E20747970653D6275B2
:1040200074746F6E2069643D636C6561722D636F9B
:104030006E666967207469746C653D22D0A3D0B444
:10404000D0B0D0BBD0B8D182D18C20D0BAD0BED025
:10405000BDD184D0B8D0B3D183D180D0B0D186D0F7
:10406000B8D18E223ED0A3D0B4D0B0D0BBD0B8D17E
:1040700082D18C20D0BAD0BED0BDD184D0B8D0B33C
:10408000D183D180D0B0D186D0B8D18E3C2F62758B
:1040900074746F6E3E3C2F6469763E3C68323ED04D
:1040A0009ED0B1D0BDD0BED0B2D0BBD0B5D0BDD0E7
:1040B000B8D0B520D184D0B0D0B9D0BBD0B020D04A
:1040C000BFD180D0BED0B3D180D0B0D0BCD0BCD115
:1040D0008B3C2F68323E3C6469763ED092D18BD0C7
:1040E000B1D0B5D180D0B8D182D0B520D184D0B0F4
:1040F000D0B9D0BB20D0BFD180D0BED0B3D180D07A
:10410000B0D0BCD0BCD18B3A3C696E707574207451
:104110007970653D66696C652069643D66696C65AA
:10412000206175746F636F6D706C6574653D6F664B
:10413000663E3C2F6469763E3C6469762069643D46
:1041400066696C652D696E666F3E3C2F6469763ECC
:104150003C6469763E3C627574746F6E207479704D
:10416000653D627574746F6E2069643D696E737429
:10417000616C6C207469746C653D22D0A3D181D1CF
:1041800082D0B0D0BDD0BED0B2D0B8D182D18C2038
:10419000D0B2D18BD0B1D180D0B0D0BDD0BDD18381
:1041A000D18E20D0BFD180D0BED0B3D180D0B0D0FE
:1041B000BCD0BCD183223ED0A3D181D182D0B0D09B
:1041C000BDD0BED0B2D0B8D182D18C20D0B2D18BEC
:1041D000D0B1D180D0B0D0BDD0BDD183D18E20D0D0
:1041E000BFD180D0BED0B3D180D0B0D0BCD0BCD1F4
:1041F000833C2F627574746F6E3E3C2F6469763E0B
:104200003C6469762069643D7374617475733E3CE7
:104210002F6469763E3C73637269707420747970A0
:10422000653D746578742F6A617661736372697035
:10423000743E2166756E6374696F6E2874297B669F
:10424000756E6374696F6E206E2872297B696628AB
:10425000655B725D2972657475726E20655B725D57
:104260002E6578706F7274733B76617220693D655C
:104270005B725D3D7B693A722C6C3A21312C65781A
:10428000706F7274733A7B7D7D3B72657475726E6C
:1042900020745B725D2E63616C6C28692E6578708A
:1042A0006F7274732C692C692E6578706F727473D9
:1042B0002C6E292C692E6C3D21302C692E6578706E
:1042C0006F7274737D76617220653D7B7D3B6E2ECF
:1042D0006D3D742C6E2E633D652C6E2E643D6675AF
:1042E0006E6374696F6E28742C652C72297B6E2E38
:1042F0006F28742C65297C7C4F626A6563742E6418
:104300006566696E6550726F706572747928742C79
:10431000652C7B636F6E666967757261626C653A66
:1043200021312C656E756D657261626C653A213064
:104330002C6765743A727D297D2C6E2E6E3D6675F4
:104340006E6374696F6E2874297B76617220653D97
:10435000742626742E5F5F65734D6F64756C653FC0
:1043600066756E6374696F6E28297B7265747572E9
:104370006E20745B2264656661756C74225D7D3AA3
:1043800066756E6374696F6E28297B7265747572C9
:104390006E20747D3B72657475726E206E2E64287B
:1043A000652C2261222C65292C657D2C6E2E6F3D9B
:1043B00066756E6374696F6E28742C6E297B7265E6
:1043C0007475726E204F626A6563742E70726F74BA
:1043D0006F747970652E6861734F776E50726F706D
:1043E000657274792E63616C6C28742C6E297D2C37
:1043F0006E2E703D222F222C6E286E2E733D30299A
:104400007D285B66756E6374696F6E28742C6E2CE4
:1044100065297B66756E6374696F6E2072287429D6
:104420007B69662832213D3D742E6C656E67746829
:104430002972657475726E206E756C6C3B76617254
:10444000206E3D7061727365496E7428742C31362C
:10445000293B72657475726E2069734E614E286EC9
:10446000293F6E756C6C3A6E7D66756E6374696F0C
:104470006E206928297B666F722876617220743DF0
:104480005B66756E6374696F6E28297B72657475DF
:10449000726E206E657720584D4C4874747052656A
:1044A00071756573747D2C66756E6374696F6E28A3
:1044B000297B72657475726E206E65772041637416
:1044C000697665584F626A65637428224D73786D0A
:1044D0006C322E584D4C4854545022297D2C667510
:1044E0006E6374696F6E28297B72657475726E20B5
:1044F0006E657720416374697665584F626A6563BB
:104500007428224D73786D6C332E584D4C4854549A
:104510005022297D2C66756E6374696F6E28297B25
:1045200072657475726E206E65772041637469766A
:1045300065584F626A65637428224D6963726F73B0
:104540006F66742E584D4C4854545022297D5D2C72
:104550006E3D21312C653D303B653C742E6C656EA3
:104560006774683B652B2B297B7472797B6E3D7475
:104570005B655D28297D63617463682872297B63AC
:104580006F6E74696E75657D627265616B7D726553
:104590007475726E206E7D66756E6374696F6E20C1
:1045A0006F2874297B72657475726E20646F6375F1
:1045B0006D656E742E676574456C656D656E7442CD
:1045C0007949642874297D66756E6374696F6E20FD
:1045D000612874297B666F7228766172206E2C6563
:1045E0003D742E73706C697428223A30323030304A
:1045F00030303422292C723D5B5D2C693D313B6E9D
:104600003D655B692B2B5D3B297B766172206F3D9D
:104610006E2E737562737472696E6728302C34293C
:104620002C613D7061727365496E74286F2C313056
:10463000293B6966282128613C3830307C7C613E0A
:1046400039303029297B76617220633D6E2E73707C
:104650006C697428225C6E22293B722E6C656E6731
:1046600074687C7C722E7075736828223A222B6FD6
:10467000293B666F7228766172206C2C753D323B47
:104680006C3D635B752B2B5D3B297B7661722073E0
:104690003D6C2E736C69636528392C2D33293B7270
:1046A0002E707573682873292C3726757C7C722EC2
:1046B0007075736828222122297D7D7D4E3D722EE2
:1046C0006A6F696E282222292C5A3D4E2E73706C17
:1046D000697428222122292E6A6F696E28222229D4
:1046E0007D66756E6374696F6E206328742C6E2905
:1046F0007B76617220653D742B322A6E2C693D6594
:104700002B312C6F3D72285A2E63686172417428D8
:1047100065292B5A2E636861724174286929293BE7
:1047200072657475726E20537472696E672E66724C
:104730006F6D43686172436F6465286F297D66758C
:104740006E6374696F6E206C28742C6E297B6E2BDF
:104750003D31323B76617220653D7B747970653AFC
:10476000742C643A7061727365496E742863286EA4
:104770002C30292B63286E2C31292C3130292C6DBB
:104780003A7061727365496E742863286E2C332900
:104790002B63286E2C34292C3130292C793A706106
:1047A000727365496E742863286E2C36292B632832
:1047B0006E2C37292B63286E2C38292B63286E2CFE
:1047C00039292C3130292C683A7061727365496E31
:1047D000742863286E2C3131292B63286E2C3132DA
:1047E000292C3130292C693A7061727365496E74D5
:1047F0002863286E2C3134292B63286E2C313529FF
:104800002C3130297D3B72657475726E20652E7473
:104810007970652B223A222B652E642E6C656164BB
:10482000696E675A65726F28292B222E222B652EFE
:104830006D2E6C656164696E675A65726F28292BED
:10484000222E222B652E792E6C656164696E675A63
:1048500065726F28292B2220222B652E682E6C650D
:104860006164696E675A65726F28292B223A222B80
:10487000652E692E6C656164696E675A65726F2872
:10488000297D66756E6374696F6E20752874297B47
:104890006F282266696C652D696E666F22292E6904
:1048A0006E6E657248544D4C3D747D66756E6374D2
:1048B000696F6E20732874297B6F2822737461746A
:1048C000757322292E696E6E657248544D4C3D7485
:1048D0002E7265706C616365282F5C6E2F67692C82
:1048E000223C6272202F3E22297D66756E637469B8
:1048F0006F6E206628297B76617220743D6F2822B6
:1049000066696C6522292E66696C65735B305D3B58
:1049100069662821742972657475726E20766F69D4
:10492000642075282222293B766172206E3D27D0B3
:1049300092D18BD0B1D180D0B0D0BD20D184D0B0B5
:10494000D0B9D0BB203C656D3E22272B742E6E6102
:104950006D652B27223C2F656D3E2C20272B28745C
:104960002E73697A652F31303234292E746F46697F
:1049700078656428292B2220D0BAD0B12E222C654C
:104980003D6E65772046696C655265616465723B72
:10499000652E726561644173546578742874292C9E
:1049A000652E6F6E6C6F61643D66756E6374696FC2
:1049B0006E2874297B6128742E7461726765742E69
:1049C000726573756C74293B76617220653D5A2E51
:1049D000696E6465784F662848292C723D5A2E69A5
:1049E0006E6465784F662858293B696628653C30B7
:1049F0007C7C723C302972657475726E2075286EED
:104A00002B223C6272202F3E3C7374726F6E673EA5
:104A1000D09DD0B5D0BAD0BED180D180D0B5D0BADB
:104A2000D182D0BDD18BD0B920D184D0B0D0B9D073
:104A3000BB20D0BFD180D0BED0B3D180D0B0D0BC4D
:104A4000D0BCD18B213C2F7374726F6E673E2229CC
:104A50002C766F6964286F2822696E7374616C6CA0
:104A600022292E7374796C652E7669736962696C7C
:104A70006974793D2268696464656E22293B7661B8
:104A80007220693D6C284F2C65292C633D6C286A87
:104A90002C72293B75286E2B223C6272202F3ED04F
:104AA0009AD0BED180D180D0B5D0BAD182D0BDD17C
:104AB0008BD0B920D184D0B0D0B9D0BB20D0BFD159
:104AC00080D0BED0B3D180D0B0D0BCD0BCD18B21EF
:104AD0003C6272202F3E3C6272202F3ED092D0B5B5
:104AE000D180D181D0B8D18F20D0BFD180D0BED0DD
:104AF000B3D180D0B0D0BCD0BCD18B20D0BAD0BE86
:104B0000D0BDD182D180D0BED0BBD0BBD0B5D180FA
:104B1000D0B03A203C7374726F6E673E222B692BC3
:104B2000223C2F7374726F6E673E2C3C6272202F92
:104B30003ED092D0B5D180D181D0B8D18F20D0BF16
:104B4000D180D0BED0B3D180D0B0D0BCD0BCD18BBE
:104B500020D0BAD0BED0BDD184D0B8D0B3D183D10B
:104B600080D0B0D182D0BED180D0B03A203C737416
:104B7000726F6E673E222B632B223C2F7374726F11
:104B80006E673E2E22292C6F2822696E7374616C29
:104B90006C22292E7374796C652E7669736962694B
:104BA0006C6974793D2276697369626C65227D7DDA
:104BB00066756E6374696F6E206428742C6E297B31
:104BC00076617220653D6928293B652E6F6E72659E
:104BD00061647973746174656368616E67653D666D
:104BE000756E6374696F6E28297B343D3D3D652E7B
:104BF00072656164795374617465262628636C65F7
:104C0000617254696D656F75742872292C6E262641
:104C10006E2829297D2C652E6F70656E2822706F95
:104C20007374222C222F222C2130292C652E73659F
:104C30007452657175657374486561646572282284
:104C4000436F6E74656E742D54797065222C2261E9
:104C500070706C69636174696F6E2F782D777777E8
:104C60002D666F726D2D75726C656E636F64656411
:104C700022292C652E73656E642874292C732822D2
:104C8000D092D18BD0BFD0BED0BBD0BDD18FD0B54C
:104C9000D182D181D18F20D0BED0BFD0B5D180D02C
:104CA000B0D186D0B8D18F2C20D0BFD0BED0B6D056
:104CB000B0D0BBD183D0B9D181D182D0B02C20D09B
:104CC000B6D0B4D0B8D182D0B52E2E2E22293B76C4
:104CD000617220723D73657454696D656F757428D7
:104CE00066756E6374696F6E28297B652E61626FCD
:104CF000727428292C732822D09AD0BED0BDD182BC
:104D0000D180D0BED0BBD0BBD0B5D18020D0BDD05B
:104D1000B520D0BED182D0B2D0B5D187D0B0D0B579
:104D2000D18222297D2C336534297D66756E6374AA
:104D3000696F6E207628742C6E297B7661722065EF
:104D40003D6928293B652E6F6E72656164797374C5
:104D50006174656368616E67653D66756E637469ED
:104D60006F6E28297B343D3D3D652E726561647907
:104D70005374617465262628636C65617254696D8D
:104D8000656F75742872292C6E26266E2829297D58
:104D90002C652E6F70656E2822676574222C222F79
:104DA0003F222B742C2130292C652E73656E6428CC
:104DB000292C732822D092D18BD0BFD0BED0BBD0AB
:104DC000BDD18FD0B5D182D181D18F20D0BED0BFFF
:104DD000D0B5D180D0B0D186D0B8D18F2C20D0BF63
:104DE000D0BED0B6D0B0D0BBD183D0B9D181D18222
:104DF000D0B02C20D0B6D0B4D0B8D182D0B52E2E21
:104E00002E22293B76617220723D73657454696D60
:104E1000656F75742866756E6374696F6E28297B7B
:104E2000652E61626F727428292C732822D09AD063
:104E3000BED0BDD182D180D0BED0BBD0BBD0B5D189
:104E40008020D0BDD0B520D0BED182D0B2D0B5D1D7
:104E500087D0B0D0B5D18222297D2C316534297D0F
:104E600066756E6374696F6E207028297B732822C3
:104E7000D09ED0BFD0B5D180D0B0D186D0B8D18FA0
:104E800020D0B2D18BD0BFD0BED0BBD0BDD0B5D09A
:104E9000BDD0B05C6ED094D0B0D0BDD0BDD0B0D1BC
:104EA0008F20D181D182D180D0B0D0BDD0B8D18671
:104EB000D0B020D0BED0B1D0BDD0BED0B2D0B8D14D
:104EC00082D181D18F20D187D0B5D180D0B5D0B754
:104ED000203520D181D0B5D0BAD183D0BDD0B42275
:104EE000292C73657454696D656F75742866756EC9
:104EF0006374696F6E28297B77696E646F772E6C97
:104F00006F636174696F6E2E72656C6F61642829BE
:104F10007D2C356533297D66756E6374696F6E20EF
:104F20007928297B732822D09ED0BFD0B5D180D0DC
:104F3000B0D186D0B8D18F20D0B2D18BD0BFD0BE67
:104F4000D0BBD0BDD0B5D0BDD0B05C6ED09FD0B5F9
:104F5000D180D0B5D0BDD0B0D0BFD180D0B0D0B28C
:104F6000D0BBD0B5D0BDD0B8D0B520D0BDD0B0204A
:104F7000D0B1D0B0D0B7D0BED0B2D18BD0B920D0C4
:104F8000B0D0B4D180D0B5D18120D0BAD0BED0BD00
:104F9000D182D180D0BED0BBD0BBD0B5D180D0B073
:104FA0002028222B502B222920D187D0B5D180D088
:104FB000B5D0B7203520D181D0B5D0BAD183D0BDFE
:104FC000D0B422292C73657454696D656F7574288B
:104FD00066756E6374696F6E28297B77696E646F7E
:104FE000772E6C6F636174696F6E3D2268747470A4
:104FF0003A2F2F222B502B222F227D2C356533293F
:105000007D66756E6374696F6E206728297B7328CF
:1050100022D09ED0BFD0B5D180D0B0D186D0B8D16B
:105020008F20D0B2D18BD0BFD0BED0BBD0BDD0B539
:10503000D0BDD0B022297D66756E6374696F6E2015
:105040006D28297B696628216F282266696C652294
:10505000292E66696C65735B305D7C7C214E2972FC
:10506000657475726E20766F696420732822D0A3F0
:10507000D0BAD0B0D0B6D0B8D182D0B520D0BAD0C6
:10508000BED180D180D0B5D0BAD182D0BDD18BD0A5
:10509000B920D184D0B0D0B9D0BB20D0BFD180D07E
:1050A000BED0B3D180D0B0D0BCD0BCD18B22293BF4
:1050B00064284D2B227B222B4E2B227D222C702903
:1050C0007D66756E6374696F6E206828297B636FD7
:1050D0006E6669726D2822D09FD0BED0B4D182D0C6
:1050E000B2D0B5D180D0B4D0B8D182D0B520D0B2B2
:1050F000D18BD185D0BED0B420D0B8D0B720D1804C
:10510000D0B5D0B6D0B8D0BCD0B020D0BED0B1D001
:10511000BDD0BED0B2D0BBD0B5D0BDD0B8D18F201D
:10512000D0BFD180D0BED0B3D180D0B0D0BCD0BCA5
:10513000D18B20D0BAD0BED0BDD182D180D0BED04C
:10514000BBD0BBD0B5D180D0B022293F6428462C3B
:1051500070293A616C6572742822D09ED0BFD0B598
:10516000D180D0B0D186D0B8D18F20D0BED182D05E
:10517000BCD0B5D0BDD0B5D0BDD0B022297D66752C
:105180006E6374696F6E206228297B766172207469
:105190003D70726F6D70742827D092D0BDD0B8D09A
:1051A000BCD0B0D0BDD0B8D0B52120D09FD180D058
:1051B000BED0B3D180D0B0D0BCD0BCD0B020D0B4A1
:1051C000D0BED180D0B0D181D187D0B5D182D0B07E
:1051D00020D0B1D183D0B4D0B5D18220D183D0B486
:1051E000D0B0D0BBD0B5D0BDD0B020D0B1D0B5D02C
:1051F000B720D0B2D0BED0B7D0BCD0BED0B6D0BD14
:10520000D0BED181D182D0B820D0B2D0BED181D190
:1052100081D182D0B0D0BDD0BED0B2D0BBD0B5D0BD
:10522000BDD0B8D18F5C6ED094D0BBD18F20D0BF11
:10523000D0BED182D0B2D0B5D180D0B6D0B4D0B5A6
:10524000D0BDD0B8D18F20D0B2D0B2D0B5D0B4D0EC
:10525000B8D182D0B520D0B220D0BFD0BED0BBD084
:10526000B520D181D0BBD0BED0B2D0BE2022D0A339
:10527000D094D090D09BD098D0A2D0AC22272C2212
:1052800022293B74262622D183D0B4D0B0D0BBD003
:10529000B8D182D18C223D3D3D742E746F4C6F7716
:1052A00065724361736528293F76286B2C67293A1C
:1052B000616C6572742822D09ED0BFD0B5D180D0E9
:1052C000B0D186D0B8D18F20D0BED182D0BCD0B5DD
:1052D000D0BDD0B5D0BDD0B022297D66756E6374C7
:1052E000696F6E207728297B76617220743D707219
:1052F0006F6D70742822D092D0BDD0B8D0BCD0B021
:10530000D0BDD0B8D0B52120D09AD0BED0BDD184E8
:10531000D0B8D0B3D183D180D0B0D186D0B8D18F1E
:1053200020D0BAD0BED0BDD182D180D0BED0BBD02B
:10533000BBD0B5D180D0B020D0B1D183D0B4D0B55E
:10534000D18220D183D0B4D0B0D0BBD0B5D0BDD025
:10535000B020D0B1D0B5D0B720D0B2D0BED0B7D069
:10536000BCD0BED0B6D0BDD0BED181D182D0B82005
:10537000D0B2D0BED181D181D182D0B0D0BDD0BE8B
:10538000D0B2D0BBD0B5D0BDD0B8D18F5C6E4950B3
:105390002DD0B0D0B4D180D0B5D18120D0BAD0BE7C
:1053A000D0BDD182D180D0BED0BBD0BBD0B5D18052
:1053B000D0B020D0B1D183D0B4D0B5D18220D183A8
:1053C000D181D182D0B0D0BDD0BED0B2D0BBD0B50B
:1053D000D0BD20D0BFD0BE20D183D0BCD0BED0BBEA
:1053E000D187D0B0D0BDD0B8D18E202D20222B5067
:1053F0002B275C6ED094D0BBD18F20D0BFD0BED134
:1054000082D0B2D0B5D180D0B6D0B4D0B5D0BDD0D6
:10541000B8D18F20D0B2D0B2D0B5D0B4D0B8D1826C
:10542000D0B520D0B220D0BFD0BED0BBD0B520D117
:1054300081D0BBD0BED0B2D0BE2022D0A3D094D0D9
:1054400090D09BD098D0A2D0AC22272C2222293BEE
:1054500074262622D183D0B4D0B0D0BBD0B8D182AC
:10546000D18C223D3D3D742E746F4C6F7765724335
:1054700061736528293F76284C2C79293A616C653F
:1054800072742822D09ED0BFD0B5D180D0B0D18642
:10549000D0B8D18F20D0BED182D0BCD0B5D0BDD0B5
:1054A000B5D0BDD0B022297D66756E6374696F6E0C
:1054B000205428297B6F2822666163746F72792DCE
:1054C0006461746122292E7374796C652E6469732A
:1054D000706C61793D22626C6F636B227D66756EC4
:1054E0006374696F6E204328297B76617220743D56
:1054F0006F2822666163746F72792D646174612D07
:10550000707722292E76616C75652C6E3D6F28228E
:10551000666163746F72792D646174612D73657255
:1055200022292E76616C75652C653D6F2822666197
:1055300063746F72792D646174612D7374722229A2
:105540002E76616C75653B69662821747C7C216EC2
:105550007C7C21652972657475726E20766F696432
:1055600020616C6572742822D094D0BED0BBD0B6B6
:10557000D0BDD18B20D0B1D18BD182D18C20D0B7EE
:10558000D0B0D0BFD0BED0BBD0BDD0B5D0BDD18BF8
:1055900020D0B2D181D0B520D0BFD0BED0BBD18F6A
:1055A0002C20D0BED0BFD0B5D180D0B0D186D0B85D
:1055B000D18F20D0BED182D0BCD0B5D0BDD0B5D097
:1055C000BDD0B022293B666F72283B6E2E6C656E93
:1055D0006774683C363B296E3D2230222B6E3B635C
:1055E0006F6E6669726D2822D09FD0BED0B4D18212
:1055F000D0B2D0B5D180D0B4D0B8D182D0B520D17E
:1056000083D181D182D0B0D0BDD0BED0B2D0BAD1FA
:105610008320D0B7D0B0D0B2D0BED0B4D181D0BA70
:10562000D0B8D18520D0B4D0B0D0BDD0BDD18BD131
:105630008522293F7628412B227B222B742B223A6C
:1056400053222B6E2B652B227D222C67293A616C0D
:105650006572742822D09ED0BFD0B5D180D0B0D191
:1056600086D0B8D18F20D0BED182D0BCD0B5D0BD2D
:10567000D0B5D0BDD0B022297D66756E6374696FD8
:105680006E207828297B76617220743D6F2822660F
:105690006163746F72792D646174612D7365722218
:1056A000293B742E76616C75653D70617273654936
:1056B0006E7428742E76616C75652C3130292B310F
:1056C0002C742E666F63757328297D66756E6374FE
:1056D000696F6E204528297B76617220742C6E2CB0
:1056E000653D646F63756D656E742E63726561747C
:1056F00065456C656D656E742822756C22293B6664
:105700006F7228652E69643D22666163746F7279D9
:105710002D737472696E67732D6C697374222C74A7
:105720003D303B6E3D535B742B2B5D3B29652E69F1
:105730006E6E657248544D4C2B3D273C6C69206958
:10574000643D22666163746F72792D737472696E41
:1057500067732D6C6973742D272B742B272220649B
:105760006174612D737472696E673D22272B6E5BC5
:10577000315D2B27223E272B6E5B305D2B223C2F89
:105780006C693E223B666F7228646F63756D656E4F
:10579000742E626F64792E617070656E64436869FF
:1057A0006C642865292C743D303B6E3D535B742B33
:1057B0002B5D3B2952286F2822666163746F7279D2
:1057C0002D737472696E67732D6C6973742D222B3F
:1057D00074292C22636C69636B222C49297D6675C0
:1057E0006E6374696F6E204928297B76617220741C
:1057F0003D746869732E676574417474726962756B
:1058000074652822646174612D737472696E6722F5
:10581000293B646F63756D656E742E626F64792EBB
:1058200072656D6F76654368696C64286F282266BF
:105830006163746F72792D737472696E67732D6C06
:105840006973742229293B766172206E3D6F28228C
:10585000666163746F72792D646174612D73747203
:1058600022293B6E2E76616C75653D742C6E2E661A
:105870006F63757328297D652831293B7661722015
:105880004D3D224669726D4845583D222C463D22C9
:1058900072756E6D61696E3D7B317D222C4C3D22AF
:1058A000436C656172436F6E66222C6B3D22436CC4
:1058B00065617243616C63222C413D2253657450D3
:1058C0003D222C483D22353334393445343433308D
:1058D0003341222C4F3D2253494E30222C583D2239
:1058E000353334393445343435373341222C6A3D2D
:1058F0002253494E57222C503D223139322E313617
:10590000382E312E32222C533D5B5B22D0A1D0B8F1
:10591000D0BDD0BAD0BED0BC2DD09432222C222CF7
:1059200044322C45322C43342C4630313034303420
:10593000303235225D2C5B22D0A1D0B8D0BDD0BA98
:10594000D0BED0BC2DD09433222C222C44332C45F5
:10595000322C43342C46303130343034303235221E
:105960005D2C5B22D0A1D0B8D0BDD0BAD0BED0BC07
:105970002DD094D09A32222C222C4B322C45322C12
:1059800043342C46303130343034303235225D2CC3
:105990005B22D0A1D0B8D0BDD0BAD0BED0BC2DD063
:1059A00094D09AD09F222C222C4D322C45312C435E
:1059B000342C547331322C547530322C4630313003
:1059C000343034303235225D2C5B22D0A1D0B8D0B7
:1059D000BDD0BAD0BED0BC2DD0942F3355222C22AE
:1059E0002C55322C45312C43322C4630313034305A
:1059F00034303235225D5D2C5A3D222C222C4E3D16
:105A000022223B4E756D6265722E70726F746F74D8
:105A10007970652E6C656164696E675A65726F3D59
:105A200066756E6374696F6E28297B726574757212
:105A30006E20746869733C31303F2230222B7468C9
:105A400069733A22222B746869737D3B76617220F8
:105A5000523D66756E6374696F6E28742C6E2C658A
:105A6000297B742E6164644576656E744C69737429
:105A7000656E65723F742E6164644576656E744C24
:105A8000697374656E6572286E2C652C2131293A14
:105A9000742E6174746163684576656E743F742E0C
:105AA0006174746163684576656E7428226F6E2236
:105AB0002B6E2C65293A745B226F6E222B6E5D3D36
:105AC000657D3B77696E646F772E46696C65262627
:105AD00077696E646F772E46696C6552656164659F
:105AE00072262677696E646F772E46696C654C69FD
:105AF00073747C7C28732822D092D0B0D18820D0B7
:105B0000B1D180D0B0D183D0B7D0B5D18020D0BDB5
:105B1000D0B520D0BFD0BED0B4D0B4D0B5D180D015
:105B2000B6D0B8D0B2D0B0D0B5D18220D0BCD0B52C
:105B3000D185D0B0D0BDD0B8D0B7D0BC20D0BFD0E8
:105B4000B5D180D0B5D0BFD180D0BED0B3D180D0B8
:105B5000B0D0BCD0BCD0B8D180D0BED0B2D0B0D044
:105B6000BDD0B8D18F20D0BAD0BED0BDD182D18027
:105B7000D0BED0BBD0BBD0B5D180D0B02E5C6E5CD7
:105B80006ED092D0BED181D0BFD0BED0BBD18CD090
:105B9000B7D183D0B9D182D0B5D181D18C20D0BE3C
:105BA000D0B4D0BDD0B8D0BC20D0B8D0B720D1812F
:105BB000D0BBD0B5D0B4D183D18ED189D0B8D18566
:105BC00020D0B1D180D0B0D183D0B7D0B5D180D0E2
:105BD000BED0B23A5C6E496E7465726E65742045D3
:105BE00078706C6F7265722031312E3020D0B82001
:105BF000D0B2D18BD188D0B52C5C6E4D6F7A696CE8
:105C00006C612046697265666F7820332E3620D02D
:105C1000B820D0B2D18BD188D0B52C5C6E476F6FD5
:105C2000676C65204368726F6D6520372E3020D019
:105C3000B820D0B2D18BD188D0B52C5C6E4F7065B6
:105C400072612031312E353020D0B820D0B2D18BC6
:105C5000D188D0B52E22292C6F282266696C652246
:105C6000292E64697361626C65643D2130292C5270
:105C7000286F282266696C6522292C226368616E70
:105C80006765222C66292C52286F2822666163746E
:105C90006F72792D646174612D73686F7722292C7E
:105CA00022636C69636B222C54292C52286F2822A2
:105CB000666163746F72792D646174612D736572AE
:105CC0002D696E6322292C22636C69636B222C7808
:105CD000292C52286F2822666163746F72792D64B3
:105CE0006174612D7374722D6C69737422292C2276
:105CF000636C69636B222C45292C52286F2822661D
:105D00006163746F72792D646174612D73656E6463
:105D100022292C22636C69636B222C43292C522884
:105D20006F2822696E7374616C6C22292C22636C5B
:105D300069636B222C6D292C52286F2822636C65B5
:105D400061722D63616C6322292C22636C69636B21
:105D5000222C62292C52286F2822636C6561722DD7
:105D6000636F6E66696722292C22636C69636B22FC
:105D70002C77292C52286F28226578697422292CC7
:105D800022636C69636B222C68297D2C66756E63B7
:105D900074696F6E28742C6E297B7D5D293B3C2FC6
:105DA0007363726970743E3C2F626F64793E3C2F5E
:105DB00068746D6C3E0000008699CE2E4B3600084C
:105DC00000000000B55D00080040404040404040F9
:105DD00040404141414141404040404040404040BE
:105DE0004040404040404040400502020202020262
:105DF00002020202020202020220202020202020B1
:105E000020202002020202020202909090909090C4
:105E10001010101010101010101010101010101082
:105E200010101010020202020202888888888888F6
:105E300008080808080808080808080808080808E2
:105E4000080808080202020240000000C95D0008BC
:105E5000485454502F312E3120323030204F4B20B7
:105E60000D0A436F6E6E656374696F6E3A20636CE2
:105E70006F73650D0A4163636573732D436F6E74B1
:105E8000726F6C2D416C6C6F772D4F726967696E04
:105E90003A2A0D0A0D0A205265616479210D0A0D16
:105EA0000A000000485454502F312E312032303037
:105EB000204F4B200D0A436F6E6E656374696F6EE1
:105EC0003A20636C6F73650D0A4163636573732DCC
:105ED000436F6E74726F6C2D416C6C6F772D4F72C7
:105EE0006967696E3A2A0D0A0D0A00000C5F000806
:105EF00000000020400200003E030008A85F0008E8
:105F000040020020308E0000C81A000811847A0375
:105F10000A0009ED010203040607080912351201FF
:105F20001B4003052A41052A42052A43052A440548
:105F30002A45052A46052A470513402082089A412A
:105F40000C9A420C9A430C9A440C9A450C9A460CB3
:105F50009A470C111209022C02232E011B0309047B
:105F60001A29041A49041A69041A89041AA9041A74
:105F7000C90422E933200A2A26052B202A0A2905EA
:105F80002B204A0A29052B206A0A29052B208A0A78
:105F900029052B20AA0A29052B20CA0A29052B200E
:085FA000EA0A2905CA09A20062
:040000050800018965
:00000001FF
